:100000000C945B000C9483000C9483000C9483008C
:100010000C9483000C9483000C9483000C94830054
:100020000C9483000C9483000C9483000C94830044
:100030000C9483000C9483000C9483000C94830034
:100040000C9470040C9483000C94F1060C948300BF
:100050000C9483000C9483000C9483000C94830014
:100060000C9483000C948300000024272A000025B0
:10007000282B000023262904040404040404040299
:100080000202020202030303030303010204081035
:100090002040800102040810200102040810200002
:1000A0000000070002010000030406000000000039
:1000B00000000000C80211241FBECFEFD4E0DEBF55
:1000C000CDBF11E0A0E0B1E0E4E3FFE002C00590A5
:1000D0000D92A836B107D9F712E0A8E6B1E001C049
:1000E0001D92A430B107E1F710E0C6EBD0E004C0E8
:1000F0002297FE010E949407C43BD107C9F70E94D2
:10010000C1020C9498070C94000040E855E260E0AE
:1001100070E086E791E00E94DC0264E670E080E037
:1001200090E00E94DB0461E0809148010E94C205DA
:1001300061E080914A010E94C20561E080914C011A
:100140000E94C20560E08EE00E94C20560E08FE080
:100150000E94C20560E080E10E94C20560E081E18A
:100160000E94C20561E08EE00E94E00561E08FE040
:100170000E94E00561E080E10E94E00561E081E12C
:100180000E94E005809168010E94500581509240D4
:100190003CF081E090E090936B0180936A0104C091
:1001A00010926B0110926A0180914E010E945005DD
:1001B000815092403CF082E090E090936D018093FA
:1001C0006C0104C010926D0110926C01809150017D
:1001D0000E945005815092403CF084E090E0909362
:1001E0006F0180936E0104C010926F0110926E0136
:1001F000809152010E945005815092403CF088E06D
:1002000090E0909371018093700104C0109271018D
:100210001092700180916C0190916D0120916A01A2
:1002200030916B01820F931F20916E0130916F010D
:10023000820F931F2091700130917101820F931FE3
:10024000909373018093720160E071E086E791E022
:100250000E94F102609172017091730186E791E052
:100260000E944004089560E0809158010E94E005DA
:1002700060E080915A010E94E00560E070E08091AA
:1002800054010E946E0560E080915C010E94E005CF
:1002900060E080915E010E94E00560E070E0809186
:1002A00056010E946E0508950F931F93CF93DF931D
:1002B0008C010E94330164E670E080E090E00E94CF
:1002C000DB0460E080915C010E94E00561E08091C8
:1002D0005E010E94E00560E0809158010E94E00507
:1002E00061E080915A010E94E005C0E4D0E011C0B5
:1002F000BE01809154010E946E05BE01809156019D
:100300000E946E0564E670E080E090E00E94DB04ED
:100310002A960C171D0764F7B801809156010E94B8
:100320006E05B801809154010E946E05DF91CF9156
:100330001F910F9108950F931F93CF93DF938C011B
:100340000E94330164E670E080E090E00E94DB04EC
:1003500061E080915C010E94E00560E080915E01B7
:100360000E94E00561E0809158010E94E00560E094
:1003700080915A010E94E005C0E4D0E011C0BE01A6
:10038000809154010E946E05BE01809156010E9429
:100390006E0564E670E080E090E00E94DB042A963F
:1003A0000C171D0764F7B801809156010E946E0575
:1003B000B801809154010E946E05DF91CF911F9189
:1003C0000F9108950F931F93CF93DF938C010E9499
:1003D000330164E670E080E090E00E94DB0461E0BD
:1003E00080915C010E94E00560E080915E010E94C6
:1003F000E00560E0809158010E94E00560E0809196
:100400005A010E94E00560E070E0809154010E9472
:100410006E05C0E4D0E00CC0BE01809156010E9480
:100420006E0564E670E080E090E00E94DB042A96AE
:100430000C171D078CF7B801809156010E946E05BC
:10044000DF91CF911F910F9108950F931F93CF9339
:10045000DF938C010E94330164E670E080E090E05D
:100460000E94DB0461E0809158010E94E00560E099
:1004700080915A010E94E00560E080915C010E9439
:10048000E00560E080915E010E94E00560E070E0C0
:10049000809156010E946E05C0E4D0E00CC0BE0100
:1004A000809154010E946E0564E670E080E090E067
:1004B0000E94DB042A960C171D078CF7B801809167
:1004C00054010E946E05DF91CF911F910F91089505
:1004D00086E791E00E94D902882309F451C086E79B
:1004E00091E00E94D6029093730180937201873548
:1004F000910551F48FEF90E00E9454016BE171E09F
:1005000086E791E00E94300380917201909173011F
:100510008A35910551F48FEF90E00E949B0162E2D1
:1005200071E086E791E00E94300380917201909122
:1005300073018134910551F48FEF90E00E94250200
:100540006CE271E086E791E00E94300380917201D5
:10055000909173018335910551F48FEF90E00E94E3
:10056000E2016BE371E086E791E00E943003809145
:100570007201909173018035910511F40E9433014D
:1005800008950E9413050E9485000E946802FDCF15
:1005900084E691E090937701809376010895862F09
:1005A0000E94B00608950E94E80608950E94C906B8
:1005B00008950E94B8060895CB01BA010E947706FB
:1005C0000895DC01ED91FC910190F081E02D0995F9
:1005D0000895DC01ED91FC910190F081E02D0995E9
:1005E00008950F931F93CF93DF938C01EB0109C004
:1005F0002196D801ED91FC910190F081E02DC80188
:10060000099568816623A1F7DF91CF911F910F9122
:1006100008950F931F938C01DC01ED91FC910190E3
:10062000F081E02D6DE00995D801ED91FC910190EC
:10063000F081E02D6AE0C80109951F910F9108959E
:100640000F931F938C01DC01ED91FC910190F081DF
:10065000E02D0995C8010E9409031F910F9108958B
:100660000F931F938C010E94F102C8010E9409039D
:100670001F910F9108950F931F938C01DC01ED9151
:10068000FC910190F081E02D0995C8010E940903B9
:100690001F910F9108952F923F924F925F926F9208
:1006A0007F928F929F92AF92BF92CF92DF92EF9202
:1006B000FF920F931F93DF93CF93CDB7DEB7A09731
:1006C0000FB6F894DEBF0FBECDBF1C016A017B01DF
:1006D000411551056105710549F4DC01ED91FC916D
:1006E0000190F081E02D60E3099554C0882499249D
:1006F0005401422E55246624772401E010E00C0FAB
:100700001D1F080D191DC701B601A30192010E940A
:100710004107F80160830894811C911CA11CB11C45
:10072000C701B601A30192010E944107C901DA0184
:100730006C017D01C114D104E104F104F1F681E002
:10074000E82EF12CEC0EFD1EE80CF91C3E0108947D
:10075000611C711CD501C4010197A109B1096C018B
:10076000C818D90814C0F601EE0DFF1D60816A306B
:1007700010F4605D01C0695CD101ED91FC910190C4
:10078000F081E02DC10109950894E108F1086E148B
:100790007F0449F7A0960FB6F894DEBF0FBECDBF19
:1007A000CF91DF911F910F91FF90EF90DF90CF904D
:1007B000BF90AF909F908F907F906F905F904F9081
:1007C0003F902F9008952AE00E944B0308950F93C5
:1007D0001F938C010E94E303C8010E9409031F912B
:1007E0000F910895AB0160E070E00E94E30308956B
:1007F0000F931F938C01AB0160E070E00E94E30354
:10080000C8010E9409031F910F910895EF92FF9272
:100810000F931F93CF93DF93EC017A018B0177FF46
:100820000FC0E881F9810190F081E02D6DE209951A
:1008300010950095F094E094E11CF11C011D111D30
:100840002AE0B801A701CE010E944B03DF91CF91AE
:100850001F910F91FF90EF9008950F931F938C01BC
:100860000E940604C8010E9409031F910F91089578
:10087000AB01662757FD6095762F0E940604089508
:100880000F931F938C01AB01662757FD6095762F60
:100890000E940604C8010E9409031F910F91089548
:1008A000DC012115310541F4ED91FC910190F081BD
:1008B000E02D642F099508952A30310519F40E941E
:1008C000060408950E944B0308950F931F938C0113
:1008D0000E945004C8010E9409031F910F910895BE
:1008E0001F920F920FB60F9211242F938F939F9305
:1008F000AF93BF938091780190917901A0917A0193
:10090000B0917B018050904CAF4FBF4F80937801E6
:1009100090937901A0937A01B0937B0127C08091D5
:10092000780190917901A0917A01B0917B01805872
:100930009E43A040B0408093780190937901A093AA
:100940007A01B0937B0180917C0190917D01A0910F
:100950007E01B0917F010196A11DB11D80937C01A4
:1009600090937D01A0937E01B0937F0180917801E7
:1009700090917901A0917A01B0917B0181589E43B9
:10098000A040B04060F6BF91AF919F918F912F91A1
:100990000F900FBE0F901F9018958FB7F89420916D
:1009A0007C0130917D0140917E0150917F018FBF8C
:1009B000B901CA010895EF92FF920F931F937B0133
:1009C0008C018FB7F89440917C0150917D0160912A
:1009D0007E0170917F018FBF2FB7F89480917C01C9
:1009E00090917D01A0917E01B0917F012FBF841B6A
:1009F000950BA60BB70B8E159F05A007B10760F3EB
:100A00001F910F91FF90EF900895019759F0FC010D
:100A1000EE0FFF1FEE0FFF1F32978FB7F89431973D
:100A2000F1F78FBF0895789484B5826084BD84B552
:100A3000816084BD85B5826085BD85B5816085BDD9
:100A4000EEE6F0E0808181608083E1E8F0E0808183
:100A500082608083808181608083E0E8F0E0808133
:100A600081608083E1EBF0E0808184608083E0EB53
:100A7000F0E0808181608083EAE7F0E0808184603B
:100A80008083808182608083808181608083808197
:100A9000806880831092C100089580936601089554
:100AA0008F70909166019295990F990F907C982B79
:100AB00090937C0080917A00806480937A0080918A
:100AC0007A0086FDFCCF2091780040917900942F28
:100AD00080E030E0282B392BC90108951F93CF9374
:100AE000DF93182FEB0161E00E94C205E12FF0E0D7
:100AF000E156FF4F8491833051F4809180008068EB
:100B000080938000D0938900C093880037C08430E0
:100B100051F480918000806280938000D0938B009C
:100B2000C0938A002BC0813029F484B5806884BDCD
:100B3000C7BD24C0823029F484B5806284BDC8BD9D
:100B40001DC0863041F48091B00080688093B00071
:100B5000C093B30013C0873041F48091B00080622D
:100B60008093B000C093B40009C0C038D10514F41C
:100B700060E001C061E0812F0E94E005DF91CF912C
:100B80001F910895282F30E0C90185579F4FFC0120
:100B9000949129583F4FF9018491882381F0E82FDF
:100BA000F0E0E859FF4FE491F0E0662329F48081FA
:100BB00090958923808308958081892B808308956F
:100BC000482F50E0CA0181569F4FFC012491CA0171
:100BD00085579F4FFC01949149585F4FFA0134911A
:100BE0003323C1F1222331F1233021F4809180009D
:100BF0008F7705C0243031F4809180008F7D809301
:100C0000800018C0213019F484B58F7704C02230D9
:100C100021F484B58F7D84BD0DC0263021F48091F0
:100C2000B0008F7705C0273029F48091B0008F7D08
:100C30008093B000E32FF0E0E359FF4FE491F0E040
:100C4000662329F48081909589238083089580818B
:100C5000892B80830895482F50E0CA0181569F4F09
:100C6000FC012491CA0185579F4FFC01949149587A
:100C70005F4FFA013491332319F420E030E035C09E
:100C8000222331F1233021F4809180008F7705C039
:100C9000243031F4809180008F7D8093800018C0D3
:100CA000213019F484B58F7704C0223021F484B543
:100CB0008F7D84BD0DC0263021F48091B0008F77E8
:100CC00005C0273029F48091B0008F7D8093B0005B
:100CD000E32FF0E0EE58FF4FE491F0E0808120E058
:100CE00030E0892311F021E030E0C9010895EF924E
:100CF000FF920F931F937B018C0122E030E040E0D4
:100D000050E00E946307205C3D4B404F5F4FCA019B
:100D1000B901A80197010E946307C901DA0101978F
:100D2000A109B109292F3A2F4B2F552747FD5A9575
:100D30000196A11DB11D2093C50081508093C40070
:100D4000E1ECF0E080818061808380818860808335
:100D50008081806880831F910F91FF90EF900895AC
:100D6000982F8091C00085FFFCCF9093C600089516
:100D7000809180019091810180589F4F2091820144
:100D800030918301821B930B60E870E00E942E0774
:100D9000089540918201509183018091800190914A
:100DA00081018417950719F42FEF3FEF0FC0FA0167
:100DB000EC57FE4F2081CA01019660E870E00E9466
:100DC0002E07909383018093820130E0C90108953A
:100DD00080918201909183019093810180938001A1
:100DE00008951F920F920FB60F9211242F933F93E5
:100DF0004F935F936F937F938F939F93AF93BF9323
:100E0000EF93FF934091C600E0918001F091810142
:100E1000CF01019660E870E00E942E079C0180914E
:100E20008201909183012817390739F0EC57FE4F62
:100E300040833093810120938001FF91EF91BF9116
:100E4000AF919F918F917F916F915F914F913F9162
:100E50002F910F900FBE0F901F90189597FB092EA2
:100E600007260AD077FD04D049D006D000201AF416
:100E7000709561957F4F0895F6F7909581959F4FF6
:100E80000895A1E21A2EAA1BBB1BFD010DC0AA1FCB
:100E9000BB1FEE1FFF1FA217B307E407F50720F0E3
:100EA000A21BB30BE40BF50B661F771F881F991F5E
:100EB0001A9469F760957095809590959B01AC01A7
:100EC000BD01CF01089597FB092E05260ED057FDD1
:100ED00004D0D7DF0AD0001C38F4509540953095E7
:100EE00021953F4F4F4F5F4F0895F6F790958095AE
:100EF000709561957F4F8F4F9F4F0895AA1BBB1B25
:100F000051E107C0AA1FBB1FA617B70710F0A61B09
:100F1000B70B881F991F5A95A9F780959095BC012A
:100F2000CD010895EE0FFF1F0590F491E02D099477
:040F3000F894FFCF63
:100F3400486F6C612C20736F7920656C20726F622E
:100F44006F74206E756D65726F20004176616E7AE4
:100F54006F00526574726F6365646F004769726FE6
:100F640020497A71756965726461004769726F20FE
:100F74004465726563686100060008000B000100A7
:100F84000200030009000A00020003000500040037
:080F940000000000CF02010083
:00000001FF
